:020000040000FA
:020000005E2878
:08000800A000030E8312A10009
:100010000C1C1E280C100B308F00DD308E003908B0
:10002000031DB9033A08031DBA033B08031DBB03B4
:100030005D1C1E28DD115D155D10DD140B1D59289A
:100040000B11DD1C5928250803192828A503592858
:100050000408A2005D1D37285D11230884002408D0
:100060000005B83003196D308100851657285D15DD
:10007000863081008512A40C031C57280830A40088
:10008000A30A23085D3A031D5728DD1950285D1582
:10009000DD155230A3000830A4000F30A50057280A
:1000A000DD105D1E54285728BC019630A50022089B
:1000B0008400210E8300A00E200E09008501073068
:1000C000990083161F309F001F308500FF2390008A
:1000D00082308100831281309F0081010B118B16C9
:1000E0008F018E010C100B308F00DD308E000B174E
:1000F0008B1783160C148312313090000130DE0010
:10010000DD01A5013D3084002A22413084002A22ED
:10011000453084002A22493084002A2234222830A3
:10012000BA005030BB007830B900BC00DD121F119E
:100130009F113D3084007521DD121F119F15413044
:1001400084007521DD121F159F1145308400752133
:10015000DD161F159F154930840075213C08031DCD
:10016000BD28BC0A4F08B2005008B3005108B400C3
:100170000830A6005D16482196283908031DDC28A2
:10018000C02149308400D421FE213208CF00330839
:10019000D0003408D1002A223422DD172230A700F3
:1001A0000930A6003D308400D421FE212A225D12B0
:1001B00048217830B90096283A08031DEF28DD1F42
:1001C000EC282430A7000930A60041308400D42157
:1001D000FE212A225D1248217830BA0096283B0879
:1001E000031D0129DD1FFF282630A7000930A600C6
:1001F00045308400D421FE212A225D124821783026
:10020000BB00851996285E1C0F29DD161F119F1152
:100210002230A7000930A6003D3084003E29DE1CB4
:100220001B29DD161F119F152430A7000930A600D9
:10023000413084003E295E1D2729DD161F159F11C0
:100240002630A7000930A600453084003E29DE1D77
:100250004629DD161F159F152230A7000830A6007D
:10026000493084003E2975213908031D33295D1664
:10027000C021D421FE212A22342248210A30B9008B
:10028000851D33290310DE190314DE0DDD128028CD
:10029000A8010030D2000A30D300A8072608D400F5
:1002A000A807270E0F39D500A80727080F39D60051
:1002B000A80732080F39D700A807330E0F39D80026
:1002C000A80733080F39D900A807340E0F39DA0010
:1002D000A80734080F39DB0028070F39DC0052303B
:1002E000A3000830A4005D1408009721031D7529A0
:1002F000A9019721031D8129A90B792997210319A8
:100300008F29AA21DD1E8A29B80A0319B70A031901
:10031000B60A7E2900000000000000007E2914308B
:10032000B5009721031D8129B50B912908006400B0
:100330009F149F1899295D1383161E088312B1001C
:10034000031D5D171E08B000031D5D1703115D1F1F
:10035000031508000408AC00033084073108800747
:10036000840330080318300F8007031CBD29840361
:10037000800A031DBD298403800A2C08840008001C
:100380003808AD003708CE003608CD001F30AD0765
:10039000031CCD29CE0A0319CD0AAD0DCE0DCD0D0E
:1003A000AD0DCE0DCD0D080003300407AC00840068
:1003B0004D08AA004E08AB00AE01AF012030B500D9
:1003C000000D8403800D8403800D8403800DAF0D28
:1003D000AE0D2C088400800D2B08AF022A08031CE8
:1003E0002A0FAE02031800140018F929AE072B08D3
:1003F000AF07B50BE029033084020800033004077F
:10040000AC00840003101030B500B201B301B40198
:100410002C088400800D8403800DB40DB30DB20D43
:10042000B50B152A023084020800343084001F22E4
:10043000333084001F22323084001F22082A033008
:100440000007AD00AD19800030300007AD00AD1BD6
:10045000800008008001840A8001840A8001840AE7
:100460008001033084020800B801B701B60108001A
:02400E00CC3FA5
:00000001FF
